:021DFE00820061
:101E0000003406340B340B340C340C340D340D34E4
:101E10000D340D340E340E340E340F340F341034B0
:101E20001034113411341134113412341234133487
:101E3000133414341434143415341534163416345D
:101E400017341734183418341834193419341A3430
:101E50001B341B341C341C341C341D341E341F34FE
:101E60001F342034203421342134223423342334C9
:101E70002334243425342634273427342734283493
:101E800029342A342B342B342B342C342D342E3457
:101E90002F342F3430343134323433343334333418
:101EA00034343534363436343734383439343A34DB
:101EB0003A343B343C343D343E343E343F34403499
:101EC0004134423442344334443445344534463456
:101ED0004734483449344A344B344C344D344D340F
:101EE0004F345034513451345234533454345534C3
:101EF00056345734583459345A345B345C345D3476
:101F00005E345F3460346134623463346434653425
:101F100066346734683469346A346B346C346D34D5
:101F20006F346F3470347234723474347534763480
:101F3000773478347A347A347C347D347E347F3428
:101F400081348234833484348534863488348934CB
:101F50008A348B348D348D348F3490349134923470
:101F60009434943496349734983499349B349C3414
:101F70009D349F34A034A134A234A334A434A634B5
:101F8000A734A834AA34AB34AC34AE34AF34B03454
:101F9000B234B334B434B634B734B834BA34BB34EE
:101FA000BD34BE34BF34C134C234C334C534C63486
:101FB000C834C934CA34CC34CD34CF34D134D1341C
:101FC000D334D434D634D834D934DB34DC34DD34AF
:101FD000DF34E034E234E334E534E734E934EB343D
:101FE000EC34EE34EF34F134F234F434F634F734C4
:101FF000F934FA34FC34FE34FF34FF34FF34FF3458
:00000001FF
